:020000040000FA
:02000000B8291D
:080008009818181218162C08B4
:10001000A0002D08A100A201A3010E280F28640052
:100020008C1A2B28FF30A207031CA307031CA00770
:10003000031CA107031C0800220F0D28230F0E2804
:10004000FA30A2000030A3000F28981818121816D2
:1000500064008C1E28281A080314B32904086400BD
:100060000C1E2F2899000314B329A401A501B31273
:10007000AE21031C0800D33E0319B3162D3EC63E25
:10008000031846280A3E031C38284D28F33E03185F
:100090003828063E031C38280A3EA2000430A3007C
:1000A000A20EA20DA40DA50DA30B5128A90303199F
:1000B0009A28AE21031C0800C63E031863280A3E96
:1000C000031C9A284D28F33E03189A28063E031C69
:1000D0009A280A3E4D28A401A501B312AE21031CA3
:1000E0000800D33E0319B3162D3EC63E03186E28F2
:1000F0000A3E031C6E28A2000310240DA000250D4B
:10010000A100200DA10DA4070318A10A2108A5072D
:10011000A40DA50D2208A4070318A50AA903031915
:100120009A28AE21031C0800C63E03189A280A3EEE
:1001300003187B28B31EA128A409A509A40A031942
:10014000A50A24080314B329B31329080319B31704
:100150000530A8002730A3001030BA200330A300D8
:10016000E830BA20A3016430BA20A3010A30BA20D3
:100170002408C128A2002508A1002408A00092217B
:100180002008A000A8030319B31329080319CB28DA
:100190002802031808002008031DB313B31B08002E
:1001A000303EAE290830A600A70037088400350885
:1001B00033192321331D2521360884008417340880
:1001C0008004A001A10126080319B329B31818213E
:1001D0003608840000083405FF3EA00DA10DB31CB5
:1001E0001821A60BE6282708331849292008B32927
:1001F0000830A60037088400350833192321331D41
:10020000252136088400841734098005260803193F
:10021000B3293318492136088400A10CA00C00082A
:100220003404031C340680001821A60B0B29B329C3
:10023000370884003508800600001E291F29202960
:1002400021298006080080042829FF3A80052929F1
:10025000FF3A84178005B329A301A200FF30A2074B
:10026000031CA307031CB3290330A100E6303A2185
:100270002E29A101FC3EA000A109031C4529FF3045
:100280000000A00703184029A0076400A10F3F2920
:100290000800A201A3015029A10CA00CA20DA30DDE
:1002A000FF3E03184C292308A1002208A000B3290F
:1002B0000310A00DA10DFF3E031858292008B329F3
:1002C0000310A10CA00CFF3E031860292008B329DD
:1002D000A101A301A20001307429A101A301A20080
:1002E00004307429A2000530A80023082102031D50
:1002F0007B29220820020430031801300319023040
:100300002805031DFF30B329A2002008A6002408F9
:10031000A0002608A4002108A6002508A1002608A0
:10032000A5009429A501A4011030A600210DA40D5B
:10033000A50D2208A4022308031C230FA5020318FD
:10034000A8292208A40723080318230FA5070310D0
:10035000A00DA10DA60B96292008B3298400310811
:100360008A0030088200831303138312640008009C
:1003700083168130990024309800831290309800C1
:10038000831607309F008117181506108614061172
:1003900086118613061386128312E90186138316CB
:1003A000861383128612831686128312061383160F
:1003B0000613413083128A012F2054308A012F20E6
:1003C00034308A012F2035308A012F2020308A01D5
:1003D0002F2053308A012F2074308A012F20613062
:1003E0008A012F2072308A012F2074308A012F2039
:1003F00069308A012F206E308A012F2067308A01F0
:100400002F202E308A012F202E308A012F202E30CF
:100410008A012F202E308A012F200D308A012F20B3
:100420000A308A012F20BE01BF01DE01C401C501CF
:10043000861583168611C83083128A012C218A11F1
:100440000A122C238A110A12212C8A110A129F22C5
:1004500086118316861106308312B6000130B4006F
:100460000630B7000430B5000130B3005E08A000CC
:10047000A1018A01F8204408A0004508A10010301D
:100480008A01F9203808A0003908A1008A01F82063
:1004900064005E08683C8A110A120319562A640037
:1004A0005E08523C8A110A12031D6D2A0630B600FE
:1004B0000130B4000630B7000430B5000130B3009D
:1004C000A001A10110308A01F920A001A101103082
:1004D0008A01F9208A110A12892A64005E08563CB2
:1004E0008A110A1203197B2A64005E08543C8A119F
:1004F0000A12031D892A0630B6000130B400063006
:10050000B7000430B5000130B300A001A1018A0199
:10051000F82008003A08A0003B08A1003C08A4000D
:100520003D08A5000130A30008308A018421C600DF
:100530002108C7002408BE002508BF0008000310DA
:10054000C40DC50D39184414391C44103808B800BE
:10055000B9010800E801E201861183168611063010
:100560008312B6000130B4000630B7000430B50085
:100570000130B3005730A000A1018A01F8200630F5
:10058000B6000230B4000630B7000430B5000230C7
:10059000B3008A01D220E700E80364006808003C49
:1005A0008A110A120319DC2A64008A110A12E71F51
:1005B000BF2A8A110A12272B41308A012F2054307A
:1005C0008A012F2034308A012F2035308A012F20D4
:1005D00044308A012F2042308A012F2030308A0196
:1005E0002F2034308A012F2031308A012F202030F3
:1005F0008A012F2042308A012F2075308A012F2056
:1006000073308A012F2079308A012F2020308A010F
:100610002F2045308A012F2072308A012F2072301E
:100620008A012F206F308A012F2072308A012F20FB
:1006300021308A012F200D308A012F200A308A01B3
:100640002F2006178316061383120130E200861549
:100650008316861183120800861183168611831271
:100660005230DE00C401C501B801B9018A0125225A
:10067000E4016400203064028A110A120318522B2C
:100680000630B6000230B4000630B7000430B500C2
:100690000230B3008A01D220DD00E40A8A110A1276
:1006A000031D392B861583168611831208008A01D3
:1006B000AA2238306705C000C1014008A0004108E7
:1006C000A10003308A016321C0002108C100A001FC
:1006D000A1014108A30040088A0172218A110A126F
:1006E000031DBD2B44308A012F2061308A012F2049
:1006F00074308A012F2061308A012F2046308A0110
:100700002F206C308A012F2061308A012F20733016
:100710008A012F2068308A012F2020308A012F2063
:1007200053308A012F2069308A012F207A308A01C4
:100730002F2065308A012F203D308A012F2035304F
:100740008A012F2031308A012F2032308A012F2058
:100750006B308A012F2062308A012F2069308A0194
:100760002F2074308A012F200D308A012F200A306B
:100770008A012F208A110A12132C0130E300013064
:10078000C0020030031C013EC1026308A000400803
:100790008A015B21E30044308A012F2061308A0105
:1007A0002F2074308A012F2061308A012F2046309B
:1007B0008A012F206C308A012F2061308A012F207E
:1007C00073308A012F2068308A012F2020308A015F
:1007D0002F2053308A012F2069308A012F207A3050
:1007E0008A012F2065308A012F203D308A012F2079
:1007F000A9016308A400A5012E30B000B1018A014F
:10080000A4206D308A012F2062308A012F206930A8
:100810008A012F2074308A012F200D308A012F2069
:100820000A308A012F2008005B08DE004608C40059
:100830004708C5003E08B8003F08B9008A012522D4
:10084000080041308A012F2074308A012F206D303A
:100850008A012F2065308A012F206C308A012F20D9
:1008600020308A012F2041308A012F2054308A0104
:100870002F2034308A012F2035308A012F20443038
:100880008A012F2042308A012F2030308A012F2008
:1008900034308A012F2031308A012F2020308A0104
:1008A0002F2044308A012F2065308A012F206D309F
:1008B0008A012F206F308A012F200D308A012F20CE
:1008C0000A308A012F203D308A012F203D308A01D5
:1008D0002F203D308A012F203D308A012F203D30CE
:1008E0008A012F203D308A012F203D308A012F20A0
:1008F0003D308A012F203D308A012F203D308A0172
:100900002F203D308A012F203D308A012F203D309D
:100910008A012F203D308A012F203D308A012F206F
:100920003D308A012F203D308A012F203D308A0141
:100930002F203D308A012F203D308A012F200D309D
:100940008A012F200A308A012F208A0157230D3077
:100950008A012F200A308A012F2041308A012F205E
:1009600074308A012F206D308A012F2065308A0172
:100970002F206C308A012F2020308A012F20443014
:100980008A012F2061308A012F2074308A012F20A4
:1009900061308A012F2046308A012F206C308A0175
:1009A0002F2061308A012F2073308A012F20683078
:1009B0008A012F2020308A012F2044308A012F20E5
:1009C00065308A012F206D308A012F206F308A0117
:1009D0002F200D308A012F200A308A012F20573016
:1009E0008A012F2061308A012F2069308A012F204F
:1009F00074308A012F2069308A012F206E308A01DD
:100A00002F2067308A012F2020308A012F20663066
:100A10008A012F206F308A012F2072308A012F2007
:100A200020308A012F2064308A012F2061308A0112
:100A30002F2074308A012F2061308A012F202E3020
:100A40008A012F202E308A012F202E308A012F205C
:100A50002E308A012F200D308A012F200A308A0182
:100A60002F204F308A012F2070308A012F207430C0
:100A70008A012F2069308A012F206F308A012F20B0
:100A80006E308A012F2073308A012F203A308A017C
:100A90002F200D308A012F200A308A012F2031307B
:100AA0008A012F2020308A012F202D308A012F200B
:100AB00020308A012F2052308A012F2065308A0190
:100AC0002F2061308A012F2064308A012F202030AE
:100AD0008A012F2066308A012F2072308A012F2050
:100AE0006F308A012F206D308A012F2020308A013B
:100AF0002F2061308A012F2064308A012F2064303A
:100B00008A012F2072308A012F2065308A012F2020
:100B100073308A012F2073308A012F200D308A0113
:100B20002F200A308A012F2032308A012F202030D6
:100B30008A012F202D308A012F2020308A012F207A
:100B400057308A012F2072308A012F2069308A01A4
:100B50002F2074308A012F2065308A012F20203009
:100B60008A012F2074308A012F206F308A012F20B4
:100B700020308A012F2061308A012F2064308A01C1
:100B80002F2064308A012F2072308A012F20653097
:100B90008A012F2073308A012F2073308A012F2081
:100BA00020308A012F2065308A012F2072308A017F
:100BB0002F2061308A012F2073308A012F20653069
:100BC0008A012F2020308A012F2066308A012F20B1
:100BD00069308A012F2072308A012F2073308A01F8
:100BE0002F2074308A012F200D308A012F200A30E7
:100BF0008A012F2033308A012F2020308A012F20B4
:100C00002D308A012F2020308A012F2057308A0171
:100C10002F2072308A012F2069308A012F207430F2
:100C20008A012F2065308A012F2020308A012F2051
:100C300074308A012F206F308A012F2020308A01E2
:100C40002F2061308A012F2064308A012F206430E8
:100C50008A012F2072308A012F2065308A012F20CF
:100C600073308A012F2073308A012F2020308A01AF
:100C70002F206E308A012F206F308A012F202030E4
:100C80008A012F2065308A012F2072308A012F209F
:100C900061308A012F2073308A012F2065308A014C
:100CA0002F200D308A012F200A308A012F20343066
:100CB0008A012F2020308A012F202D308A012F20F9
:100CC00020308A012F2057308A012F2072308A016C
:100CD0002F2069308A012F2074308A012F2065303F
:100CE0008A012F202F308A012F2052308A012F2095
:100CF00065308A012F2061308A012F2064308A01FB
:100D00002F2020308A012F2054308A012F20653077
:100D10008A012F2073308A012F2074308A012F20FE
:100D200020308A012F2061308A012F2074308A01FF
:100D30002F2020308A012F2061308A012F2064303B
:100D40008A012F2064308A012F2072308A012F20DF
:100D500065308A012F2073308A012F2073308A0179
:100D60002F200D308A012F200A308A012F200D30CC
:100D70008A012F200A308A012F2041308A012F203A
:100D800064308A012F2064308A012F2072308A015A
:100D90002F2065308A012F2073308A012F20733075
:100DA0008A012F2020308A012F206D308A012F20C8
:100DB00075308A012F2073308A012F2074308A0108
:100DC0002F2020308A012F2062308A012F206530A9
:100DD0008A012F2020308A012F2061308A012F20A4
:100DE00020308A012F2064308A012F206F308A0141
:100DF0002F2075308A012F2062308A012F206C301D
:100E00008A012F2065308A012F2020308A012F206F
:100E100077308A012F206F308A012F2072308A01AB
:100E20002F2064308A012F2020308A012F20693042
:100E30008A012F206E308A012F2020308A012F2036
:100E400068308A012F2065308A012F2078308A018E
:100E50002F200D308A012F200A308A012F20543094
:100E60008A012F2068308A012F2065308A012F20C7
:100E700020308A012F207E308A012F2020308A01E5
:100E80002F2028308A012F2074308A012F206930CA
:100E90008A012F206C308A012F2064308A012F2094
:100EA00065308A012F2029308A012F2020308A01C5
:100EB0002F2069308A012F2073308A012F202030A3
:100EC0008A012F2075308A012F2073308A012F204C
:100ED00065308A012F2064308A012F2020308A015A
:100EE0002F2061308A012F2073308A012F2020307B
:100EF0008A012F2061308A012F2020308A012F2083
:100F000073308A012F2074308A012F2061308A01CA
:100F10002F2072308A012F2074308A012F202F3029
:100F20008A012F2073308A012F2074308A012F20EC
:100F30006F308A012F2070308A012F2020308A01E3
:100F40002F2063308A012F206F308A012F206430D8
:100F50008A012F2065308A012F200D308A012F2031
:100F60000A308A012F2066308A012F206F308A01D3
:100F70002F206C308A012F206C308A012F206F3097
:100F80008A012F2077308A012F2065308A012F2097
:100F900064308A012F2020308A012F2062308A019C
:100FA0002F2079308A012F2020308A012F207430A1
:100FB0008A012F2068308A012F2065308A012F2076
:100FC00020308A012F206F308A012F2070308A0153
:100FD0002F2074308A012F2069308A012F206F3032
:100FE0008A012F206E308A012F2020308A012F2085
:100FF00061308A012F206E308A012F2064308A01EF
:101000002F2020308A012F2074308A012F20683051
:101010008A012F2065308A012F2020308A012F205D
:1010200061308A012F2064308A012F2064308A01C8
:101030002F2072308A012F2065308A012F207330D3
:101040008A012F2073308A012F200D308A012F2032
:101050000A308A012F2045308A012F2078308A01FA
:101060002F2061308A012F206D308A012F207030AF
:101070008A012F206C308A012F2065308A012F20B1
:101080003A308A012F2020308A012F207E308A01B9
:101090002F2031308A012F2030308A012F2030302C
:1010A0008A012F2030308A012F2034308A012F20EE
:1010B00032308A012F2030308A012F2030308A01CF
:1010C0002F2030308A012F200D308A012F200A3046
:1010D0008A012F2077308A012F2069308A012F2042
:1010E0006C308A012F206C308A012F2020308A0139
:1010F0002F2072308A012F2065308A012F20613025
:101100008A012F2064308A012F2020308A012F206D
:1011100064308A012F2061308A012F2074308A01C7
:101120002F2061308A012F2020308A012F20623049
:101130008A012F2065308A012F2067308A012F20F5
:1011400069308A012F206E308A012F206E308A018B
:101150002F2069308A012F206E308A012F206730BE
:101160008A012F2020308A012F2061308A012F2010
:1011700074308A012F2020308A012F2068308A01A4
:101180002F2065308A012F2078308A012F202030CF
:101190008A012F2030308A012F2030308A012F2001
:1011A00030308A012F2034308A012F2032308A01DA
:1011B0002F2030308A012F2030308A012F2030300C
:1011C0008A012F200D308A012F200A308A012F201A
:1011D0008A0125207E3C8A150A12031DE828013069
:1011E000A9002530B000B1018A016B20E500043070
:1011F000A9002530B000B1018A013520BA002508C8
:10120000BB000430A9002530B000B1018A013520AF
:10121000BC002508BD008A018A220A308A012F20DD
:101220000D308A012F2050308A012F2061308A0131
:101230002F2067308A012F2065308A012F203A3015
:101240008A012F20A9014608A4004708A5002E30D6
:10125000B000B1018A01A42020308A012F20413042
:101260008A012F2064308A012F2064308A012F20C8
:1012700072308A012F203A308A012F20A9013E08BE
:10128000A4003F08A5002E30B000B1018A01A420BF
:101290000D308A012F200A308A012F206400650852
:1012A000013C8A150A120319992964006508023C59
:1012B0008A150A1203194A2A64006508033C8A1534
:1012C0000A1203194A2A64006508043C8A150A12A6
:1012D0000319072B4F308A012F2070308A012F20ED
:1012E00074308A012F2069308A012F206F308A01E3
:1012F0002F206E308A012F2020308A012F20453088
:101300008A012F2072308A012F2072308A012F200B
:101310006F308A012F2072308A012F2021308A01FC
:101320002F200D308A012F200A308A012F208A01B8
:10133000A72C5230DE004608C4004708C5003E080E
:10134000B8003F08B9008A0125220D308A012F20FC
:101350000A308A012F2050308A012F2061308A0103
:101360002F2067308A012F2065308A012F203A30E4
:101370008A012F20A9014608A4004708A5002E30A5
:10138000B000B1018A01A4200D308A012F200A305B
:101390008A012F200130E4000630B6000230B4008C
:1013A0000630B7000430B5000230B3008A01D22005
:1013B000DD00640080305D028A150A12031CE229F8
:1013C0002E30DD00640020305D028A150A120318F9
:1013D000EB292E30DD005D088A012F20E40A8A15F2
:1013E0000A12031DCC298615831686110D3083122F
:1013F0008A012F200A308A012F204D308A012F20A8
:101400006F308A012F2072308A012F2065308A01C7
:101410002F203F308A012F2020308A012F203130A9
:101420008A012F203D308A012F2079308A012F2018
:1014300065308A012F2073308A012F2020308A01E5
:101440002F2032308A012F203D308A012F206E302C
:101450008A012F206F308A012F200D308A012F2022
:101460000A308A012F200130A9002530B000B101D7
:101470008A016B20DD0064005D08013C8A110A12BC
:10148000031DA72CC60A0319C70A8A150A1299292F
:101490008A01A72C45308A012F206E308A012F2027
:1014A00074308A012F2065308A012F2072308A0122
:1014B0002F2020308A012F2074308A012F206530A0
:1014C0008A012F2078308A012F2074308A012F2042
:1014D00020308A012F207E308A012F2020308A017F
:1014E0002F2028308A012F2074308A012F20693064
:1014F0008A012F206C308A012F2064308A012F202E
:1015000065308A012F2029308A012F2020308A015E
:101510002F2074308A012F206F308A012F20203035
:101520008A012F2065308A012F206E308A012F20FA
:1015300064308A012F200D308A012F200A308A0161
:101540002F208430DE003E08B8003F08B9008A0131
:101550002522E830AC000330AD008A0104208A1552
:101560000A12031CA92ADD005D08A00020308A01B0
:101570006D21C8005D08A0007F308A016821CA0083
:1015800048084A048A150A12031DA92A64005D0846
:101590007E3C8A150A120319DF2A0630B600013094
:1015A000B4000630B7000430B5000130B3005D0868
:1015B000A000A1018A01F8208A150A12A92A86151D
:1015C00083168611640083126508023C8A150A128C
:1015D000031DEC2A8330DE0064006508033C8A1595
:1015E0000A12031DF52A8830DE004608C4004708A9
:1015F000C5008A01252286158316861183128A0169
:10160000AA2286158316861183128A01A72C5730C9
:101610008A012F2072308A012F2069308A012F2001
:1016200074308A012F2069308A012F206E308A01A0
:101630002F2067308A012F2020308A012F2073301D
:101640008A012F2061308A012F206D308A012F20DE
:1016500070308A012F206C308A012F2065308A017A
:101660002F2020308A012F2074308A012F206530EE
:101670008A012F2078308A012F2074308A012F2090
:1016800020308A012F2074308A012F206F308A0188
:101690002F2020308A012F2042308A012F207530E0
:1016A0008A012F2066308A012F2066308A012F2080
:1016B00065308A012F2072308A012F2020308A0164
:1016C0002F2031308A012F203A308A012F20A901A2
:1016D0004608A4004708A5002E30B000B1018A01D9
:1016E000A42020308A012F2061308A012F207430FD
:1016F0008A012F2020308A012F2041308A012F209B
:1017000064308A012F2064308A012F2072308A01D0
:101710002F2065308A012F2073308A012F207330EB
:101720008A012F203A308A012F20A9013E08A40007
:101730003F08A5002E30B000B1018A01A4200D3071
:101740008A012F200A308A012F208430DE003E08D3
:10175000B8003F08B9008A0125223E30C200C3010B
:10176000E4016408A000A1014308A30042088A0123
:101770006A218A150A12031D282C64083F3C8A1529
:101780000A12031C112C8A150A12CA23DD008A15BD
:101790000A12112C0B308A006408D13E03188A0A01
:1017A0008200573465346C3463346F346D3465347F
:1017B0002134203454346834693473342034693427
:1017C0007334203461346E342034413474346D34D5
:1017D00065346C3420344134543434343534443436
:1017E00042343034343431344234203434346D347F
:1017F0006234693474342034643461347434613450
:1018000066346C34613473346834203438342034B2
:10181000703469346E34203463346834693470341D
:1018200021340630B6000130B4000630B700043071
:10183000B5000130B3005D08A000A1018A01F820C5
:101840005D088A012F20E40A8A150A12031DB12BB4
:101850008615831686110D3083128A012F200A30D7
:101860008A012F2052308A012F2065308A012F20D3
:1018700061308A012F2064308A012F2069308A016B
:101880002F206E308A012F2067308A012F202030D0
:101890008A012F2062308A012F2061308A012F2097
:1018A00063308A012F206B308A012F2020308A017B
:1018B0002F2062308A012F2075308A012F20663058
:1018C0008A012F2066308A012F2065308A012F205F
:1018D00072308A012F202E308A012F202E308A016B
:1018E0002F202E308A012F200D308A012F200A3020
:1018F0008A012F205430DE003E08B8003F08B900AE
:101900008A012522E4016408A000A1014308A30084
:1019100042088A016A218A150A12031DA42C063086
:10192000B6000230B4000630B7000430B500023013
:10193000B3008A01D220DD005D088A012F20E40A6D
:101940008A150A12031D832C8615831686110D3005
:1019500083128A012F200A308A012F2045308A0104
:101960002F2072308A012F2061308A012F2073309E
:101970008A012F2065308A012F2020308A012F20F4
:1019800026308A012F2020308A012F2077308A01CB
:101990002F2072308A012F2069308A012F20743065
:1019A0008A012F2065308A012F2020308A012F20C4
:1019B00074308A012F206F308A012F2020308A0155
:1019C0002F2044308A012F2061308A012F2074306B
:1019D0008A012F2061308A012F2046308A012F2072
:1019E0006C308A012F2061308A012F2073308A01E8
:1019F0002F2068308A012F2020308A012F20733059
:101A00008A012F2065308A012F2063308A012F2020
:101A100074308A012F206F308A012F2072308A01A2
:101A20002F202E308A012F202E308A012F202E3099
:101A30008A012F200D308A012F200A308A012F20A1
:101A40008330DE004608C4004708C5008A0125220D
:101A500086158316861183128A01AA22861583169B
:101A60008611831252308A012F2065308A012F207F
:101A700061308A012F2064308A012F2069308A0169
:101A80002F206E308A012F2067308A012F202030CE
:101A90008A012F2062308A012F2061308A012F2095
:101AA00063308A012F206B308A012F2020308A0179
:101AB0002F2044308A012F2061308A012F2074307A
:101AC0008A012F2061308A012F2046308A012F2081
:101AD0006C308A012F2061308A012F2073308A01F7
:101AE0002F2068308A012F2020308A012F20733068
:101AF0008A012F2065308A012F2063308A012F2030
:101B000074308A012F206F308A012F2072308A01B1
:101B10002F202E308A012F202E308A012F202E30A8
:101B20008A012F200D308A012F200A308A012F20B0
:101B30005230DE004608C4004708C5003E08B80021
:101B40003F08B9008A012522E4016408A000A10130
:101B50004308A30042088A016A218A150A12031D5C
:101B6000C62D0630B6000230B4000630B70004308F
:101B7000B5000230B3008A01D220DD005D088A0181
:101B80002F20E40A8A150A12031DA52D8615831637
:101B900086110D3083128A012F200A308A012F20EE
:101BA00046308A012F2069308A012F206E308A0149
:101BB0002F2069308A012F2073308A012F2068304E
:101BC0008A012F2065308A012F2064308A012F205E
:101BD0000D308A012F200A308A012F208A01A72C7C
:101BE00064008A150A12F02D63008A150A12F42D7A
:02400E00753FFC
:00000001FF
